:020000040000FA
:1000000080260020F9020000010300000303000025
:1000100005030000070300000903000000000000C2
:100020000000000000000000000000000B030000C2
:100030000D030000000000000F030000110300008A
:100040001303000013030000E50600001303000083
:100050001303000013030000130300001303000048
:100060001303000013030000130300001303000038
:1000700013030000A103000013030000130300009A
:100080001303000013030000130300001303000018
:100090001303000013030000130300001303000008
:1000A00013030000130300001303000013030000F8
:1000B0001303000013030000000000000000000014
:1000C00013030000130300001303000013030000D8
:1000D00013030000130300001303000000000000DE
:1000E0000000000000000000000000000000000010
:1000F0000000000000000000000000000000000000
:1001000000000000000000000000000000000000EF
:1001100000000000000000000000000000000000DF
:1001200000000000000000000000000000000000CF
:1001300000000000000000000000000000000000BF
:1001400000000000000000000000000000000000AF
:10015000000000000000000000000000000000009F
:10016000000000000000000000000000000000008F
:10017000000000000000000000000000000000007F
:10018000000000000000000000000000000000006F
:10019000000000000000000000000000000000005F
:1001A000000000000000000000000000000000004F
:1001B000000000000000000000000000000000003F
:1001C000000000000000000000000000000000002F
:1001D000000000000000000000000000000000001F
:1001E000000000000000000000000000000000000F
:1001F00000000000000000000000000000000000FF
:10020000DFF80CD000F0BAF800480047C10B00003E
:100210008026002030B4044654E8000F0D4644E820
:100220000053002BF8D1156030BC704730B4044641
:1002300054E8000F40EA010544E80053002BF7D1D1
:10024000156030BC704730B4044654E8000F00EA33
:10025000010544E80053002BF7D1156030BC70470E
:1002600030B4044654E8000F80EA010544E8005326
:10027000002BF7D1156030BC704730B4044654E809
:10028000000F00EB010544E80053002BF7D1156087
:1002900030BC704730B4044654E8000FA0EB0105B1
:1002A00044E80053002BF7D1156030BC704770B4A0
:1002B00004464FF0000054E8006F0D68AE4207BFDF
:1002C00044E80023012044E800630E60002B1CBFBB
:1002D0000020F0E770BC704730B4044654E8000FCB
:1002E00088422CBF451A054644E80053002BF5D13F
:1002F000156030BC7047000006488047064800473C
:10030000FEE7FEE7FEE7FEE7FEE7FEE7FEE7FEE7C5
:10031000FEE7FEE7C9030000010200000048704745
:10032000E026000040EA01039B0703D009E008C96A
:10033000121F08C0042AFAD203E011F8013B00F8AA
:10034000013B521EF9D27047D2B201E000F8012BF6
:10035000491EFBD270470022F6E710B513460A4645
:1003600004461946FFF7F0FF204610BD421C10F866
:10037000011B0029FBD1801A70470000064C074D75
:1003800006E0E06840F0010394E807009847103465
:10039000AC42F6D3FFF738FF94270000B4270000E3
:1003A000064882B00021016000680090044800689F
:1003B0000449C0B2496802B00847000000D10040BB
:1003C00008D5004018000020F0B5B5480023021DF4
:1003D0000178101D01254FF0805406290BD11678A5
:1003E000360708D10678C6F30316032E06D0042E6E
:1003F00004D0052E02D0062907D00EE0B4F82463FD
:10040000A84FC6F304263E6002E01678360704D1F2
:100410000678C6F30316032E02D0062904D00FE097
:10042000A24FA14E7E670EE01678360708D10678F7
:10043000C6F30316032E06D0042E04D0052E02D0D8
:10044000062907D00EE0D4F84462994FC6F342362D
:100450003E6002E01678360704D10678C6F303162C
:10046000032E02D0062906D011E0924E376827F0FD
:10047000807737600EE01678360708D10678C6F325
:100480000316032E06D0042E04D0052E02D0062912
:100490000AD011E04FF08046C6F80C31C6F8103192
:1004A000834E361F336002E01678360704D1067893
:1004B000C6F30316032E02D0062905D00CE07C4FAC
:1004C000032664373E600AE01678360704D10678C2
:1004D000C6F30316032E02D006290DD014E0764F82
:1004E00005263E60744E78363560734E08363360AC
:1004F0003F263F1D3E6002E01678360704D106789D
:10050000C6F30316052E02D0062957D062E06B4EC3
:1005100036686B4F3E60694E361D36683F1D3E6043
:10052000664E083636683F1D3E60644E0C363668AF
:100530003F1D3E60614E103636683F1D3E605F4E87
:10054000143636683F1D3E605C4E183636685C4F88
:1005500020373E60594E1C3636683F1D3E60574E70
:10056000203636683F1D3E60544E243636683F1DA7
:100570003E60524E283636683F1D3E604F4E2C3648
:1005800036683F1D3E604D4E303636684C4F403722
:100590003E604A4E343636683F1D3E60474E383620
:1005A00036683F1D3E60454E3C3636683F1D3E6016
:1005B000424E403636683F1D3E6002E016783607F0
:1005C00008D10678C6F30316032E06D0042E04D0F5
:1005D000052E02D0062907D019E0D4F85812394A5E
:1005E00001F04F01116002E0117809070FD1007886
:1005F000C0F30310032803D0042801D0052806D136
:1006000031480168C90702D06FF001010160D4F8D8
:100610003001062808D1D4F83401062804D12B482B
:10062000016841F48061016022487438016841F436
:1006300070010160BFF34F8FBFF36F8F4FF0102138
:10064000D1F80002002803DBD1F80402002822DAE6
:100650001F4A15601F480468002CFCD01524C1F8FF
:1006600000420568002DFCD0C1F804420168002951
:10067000FCD0136001680029FCD0BFF34F8F0D48F8
:10068000F0380168144A01F4E06111430160BFF3DE
:100690004F8F00BFFDE7124910480860F0BD000011
:1006A000E00F00F0403501400DF0ADBA00C007404A
:1006B0003C050040FCED00E0105600400404001032
:1006C00020C50040E40E0040000400403C170040FC
:1006D00004E5014000E401400400FA050090D00365
:1006E000980000200148006800470000100000202A
:1006F00002E008C8121F08C1002AFAD170477047EB
:10070000002001E001C1121F002AFBD17047000048
:1007100072B601F021F800BF00F020FE0028FBD1E6
:10072000104C0121208801EB00400FA100F076FF62
:1007300010480068C00700D000BE2088022101EBED
:1007400000400DA100F06AFFBFF34F8F0948E43865
:1007500001680D4A01F4E06111430160BFF34F8F5E
:1007600000BFFDE7B8000020466174616C2065722F
:10077000726F7200F0ED00E053797374656D207252
:1007800065736574000000000400FA050EB50021D1
:100790000091CDE901106A4644F20100FFF7B8FF6D
:1007A0000EBD00F003B800F009B8000072B60248B0
:1007B0000168491C01607047200000200349086857
:1007C000401E086000D162B6704700002000002083
:1007D0002DE9F041064608680C46411C4FF0A04741
:1007E0004FF0010506D005FA00F1C7F8081520689A
:1007F00000F0C8FC6068411C02D0002100F0B0FC91
:100800003168A069C1F82405607D227D31681043FC
:10081000C1F86C05D4E900123068C0F81425C0F89E
:100820000C15207D012815D1A068411C02D00021A3
:1008300000F096FCE068411C05D08540C7F80855DB
:10084000E06800F09FFCD4E902123068C0F8082587
:10085000C0F81015BDE8F0812DE9F04106460868A2
:100860000C46411C4FF0A0474FF0010506D005FA99
:1008700000F1C7F80815206800F08EFC6068411C84
:1008800002D0002100F075FC3168A069C1F8240590
:10089000607D217D32680843C2F86C05D4E90012FE
:1008A0003068C0F80C15C0F81425207D012815D13A
:1008B000A068411C02D0002100F05BFCE068411CF4
:1008C00005D08540C7F80855E06800F065FCD4E91C
:1008D00002123068C0F80825C0F81015BDE8F08194
:1008E0002DE9F0470546861C90460F464FF001095A
:1008F0000020FFF756FF1B4C20683860D4E9000148
:10090000401AA16804F21C47081A0EE0012138467B
:1009100000F018FA00F006F90146384600F012FA25
:10092000D4E90001401AA168081A401C8642EDD89B
:10093000B8F1000F03D0052065F3891002E006200E
:1009400065F39F50A2682168114004EB8101C860E3
:100950002068304420600020FFF725FF4846BDE8AE
:10096000F08700005C02002030B482680468531CE9
:100970008360A154D0E901128A4202D330BC00F056
:10098000C0BA30BC70470000034803C8814201D19F
:1009900001207047002070475C02002010B5002144
:1009A000024800F0DAF980F3100010BD780600204C
:1009B0002DE9FC5F0E008346DDE90C47C6F100001F
:1009C00098469246814600D40846012503E000BFC0
:1009D00090FBFAF06D1C5045FADAA84500D945465F
:1009E00024B1002E01DB780700D5641EB80702D5BC
:1009F000B8F1000F0AD0F80708D13CB1A54205D2E2
:100A000020215846641EFFF7AFFFF6E7002E02DAFA
:100A10004E462D2102E0780703D52B215846FFF7DB
:100A2000A3FF07F0030002280BD1B8F1000F08D193
:100A30003CB1A54205D230215846641EFFF794FF11
:100A4000F6E7CDE90047434652463146584601F0A5
:100A500081FDBDE8FC9F000070B50D4604460068AE
:100A60004FF4887100F0FEFF4FF49071206800F0A1
:100A7000F9FF4FF49271206800F0F4FF4FF4A27177
:100A8000206800F0EFFF20681249C0F804132068C6
:100A90006907000B40B2090E002806DA00F00F00CB
:100AA00000F1E02080F8141D03E000F1E02080F860
:100AB000001420680121000B40B200F01F02914099
:100AC0004009800000F1E020C0F88012C0F8001159
:100AD00070BD000010030200024600201268930758
:100AE00002D0530702D47047500714D502F0030018
:100AF000012802D002280CD105E0C2F383100B6854
:100B0000801C184404E00223086803EB925210444E
:100B1000086001207047086800EB9253C2F3891007
:100B2000401CEEE72DE9FF410026234800F007F9BD
:100B30002148001F074600F002F9204C6068009031
:100B4000A56800E000986946284004EB80000C305E
:100B5000FFF7C2FF0028F5D101AA009901EA0503B9
:100B600004EB8303491CDB6842F82030401C0091F1
:100B70000228F2D3019800F0030001280BD00228CC
:100B800010D10198032101EB90500099BDF80A6043
:100B900001EB900005E00198BDF80A60C0F38310F6
:100BA00008440090384600F0C7F808B1009860602B
:100BB00004B03046BDE8F081740600205C020020DD
:100BC00086B04FF40041002000F082FD08B1FFF72D
:100BD000DDFD00F0B5FB002000F026F908B1FFF7BD
:100BE000D5FD1F4D03241FA1288804EB004000F011
:100BF00015FDA8466E46102504A800F00BF99DF8D7
:100C00001000102800D805462946304600F02AF981
:100C100008B1FFF7BBFDB8F800002E46454604EBCF
:100C2000004016A100F0FAFC2888324604EB004090
:100C3000694600F09FFC28880FA104EB004000F0FB
:100C4000EDFC00BF00F08AFB0028FBD10F4D6426AD
:100C50004FF47A47691C38468847761EFAD1C9E7AF
:100C6000B8000020524E47206578616D706C652099
:100C7000737461727465642E0000000052616E64CA
:100C80006F6D20566563746F723A00001026000085
:100C90002DE9F047C7880446181D16468946B0FB63
:100CA000F7F1B0FBF7F207FB12009A193A44D21C95
:100CB000B2FBF7F2DDF820A001E02468491E00290C
:100CC000FBD13D1A8846B54216D818E0BAF1000F9C
:100CD00005D0211809EB08002A46091D04E020442C
:100CE00009EB08012A46001DFFF71CFB00202468C1
:100CF000761BA844B74201D9354600E03D46002E98
:100D0000E4D1BDE8F087000030B5024659B100F0EB
:100D10000BFD0021074C09E004EB810315685B889B
:100D2000AB4202D11160002030BD491C8142F3D397
:100D3000052030BD9C000020002100F009B80121F1
:100D400000F010B808B56A46FFF797FA009808BD9A
:100D500008B56A46FFF777FA08BD08B56A46FFF797
:100D600059FA08BD08B56A46FFF760FA009808BD51
:100D700008B56A46FFF78EFA009808BD70B50446BC
:100D800000252846FFF70DFD21686268086890423B
:100D90000ED9401E08600178A38AE26801FB032592
:100DA000227A2168101AC0B20A79824200D20871F0
:100DB0000020FFF7F8FC284670BD70B505460C46CC
:100DC0000020FFF7EEFCE868A98A201AB0FBF1F1D9
:100DD0002A681068431C13600170BDE87040002051
:100DE000FFF7E1BC10B530B1017A42680368891A97
:100DF000C9B21A6006E00E2010BD03681A68541CC0
:100E00001C601170491EC9B2F7D20068002101713F
:100E1000084610BD10B50446024800F0FFFD2070E2
:100E200010BD00000C28000070B50B4C217809B1F2
:100E3000852070BD00B9094809490088A4F801005F
:100E4000601C00F04FFE0500F3D100F079FE012098
:100E50002070284670BD000000000020162600000B
:100E6000C51A00000A4610B50146044800F0B9FD55
:100E7000044600F065FE204610BD00000C2800006E
:100E8000F0B505460478154889B0164640F8242088
:100E9000124A0869121DA2F1080742F82400487F8F
:100EA000385520226846FFF73DFA04942878385CCC
:100EB00048B10EB10A4A00E000226946281D00F040
:100EC0008FFF09B0F0BD0EB1064A00E0002269466E
:100ED00005F10C0000F056FEF3E7000008000020CA
:100EE000312400007D2200000FB408B503990029C9
:100EF00004D004AA00926A4600F00FF801B05DF831
:100F000014FB10B582680446002A05D0D4E9040316
:100F1000216898470020A06010BD2DE9FC4791464C
:100F20000C00804676D014F8011B39B125290ED06B
:100F30004046FFF719FD20780028F4D198F80C00FE
:100F4000002867D04046BDE8FC47FFF7DABF002025
:100F5000012221782B291BD02D2902D0302908D13C
:100F600002E040F0010001E040F00200641C002AB1
:100F7000EFD100252A290ED02178A1F130020A2ACA
:100F800011D205EB850201EB4205641C303DF1E70F
:100F900040F00400EAE7D9F800100B1DC9F8003052
:100FA0000968641C0D44217800232E290BD114F804
:100FB000011FA1F130020A2A05D203EB830201EBE3
:100FC0004203303BF3E76C290DD068290BD0692927
:100FD00021D00BDC252918D0582931D063290ED017
:100FE000642915D117E014F8011FECE7702969D0C6
:100FF000732932D075291BD0782909D120E0D9F87E
:101000000000011DC9F8001001784046FFF7ACFC54
:10101000641C90E76CE0D9F800100A1DC9F80020A4
:101020000968CDE900500A224046FFF7C1FCEFE70E
:10103000D9F800100A1DC9F8002009680A2206E044
:10104000D9F800100A1DC9F8002009681022CDE95E
:101050000050404601F07EFADAE7D9F80010002788
:101060000A1DC9F800200E68C00705D112E04046ED
:10107000761C7F1CFFF778FC31780029F7D104E05B
:10108000202140466D1EFFF76FFCBD42C0D9002DE8
:10109000F6D1BDE74EB13046FFF768F9074604E0E8
:1010A000202140466D1EFFF75FFCBD4206D9002D92
:1010B000F6D103E04046761CFFF756FC3178002954
:1010C000F8D1A5E7D9F80000011DC9F8001005689E
:1010D00030214046FFF748FC78214046FFF744FCAA
:1010E00008200021CDE90001034610222946B0E77F
:1010F000BDE8FC8770B541EA4201DDE904564FF0D6
:10110000A04441EA830141EA052104EB800041EA61
:101110000641C0F8001770BD70B541EA4201DDE933
:1011200004564FF0A04441EA830141EA052104EB53
:10113000800041EA0641C0F8001770BD1CB50021CF
:1011400000910B4601220191FFF7D4FF1CBD1CB595
:10115000002100910B4601220191FFF7DDFF1CBD2C
:101160001CB500220B46009211460192FFF7C2FF08
:101170001CBD1CB500220B46009211460192FFF7E0
:10118000CBFF1CBD1CB5002100910B460122019133
:101190001146FFF7AFFF1CBD1CB5002100910B46A7
:1011A000012201911146FFF7B7FF1CBD30B5124B6C
:1011B00001460020D3F81044224609E0157A854202
:1011C00005D1401C0A28F7DB4FF0FF3030BD5268D4
:1011D000002AF3D1421CF9D00872D3F810242AB1A6
:1011E00052684A60D3F81024516030BD0022C3F821
:1011F00010144A6030BD00005C020020F0B595B0CC
:101200001C4615460F4608461A9E00F05DFB182145
:1012100009A8FFF7A0F80E96CDE90954002308228B
:1012200003A9384600F065FB05980690BDF810004C
:10123000ADF81C00BDF81200ADF81E0000208DF8BE
:1012400021000398082600F00300012802D002289C
:1012500018D032E003983346850AC0F3C2008DF8F7
:10126000200003980FA9C0F38314A200384600F0B1
:1012700040FB09A8009006AB22460FA9284600F0C3
:101280007FFA1AE00398840DC0F3C2008DF82000A5
:10129000082C01D2254600E0082533462A460FA92E
:1012A000384600F026FB2E44641B09AB06AA2946EB
:1012B0000FA800F0B7F9002CEAD1384600F00AFB7D
:1012C00015B0F0BD7047012000F0F6BF084810B51A
:1012D0000178084A515C19B1001D00F00DFE02E0D2
:1012E0000C3000F01BFDBDE81040002000F0E4BF12
:1012F000280000200400002008B5034A0092402383
:10130000024AFFF77BFF08BD752100005C01002049
:101310000A4A012902EBC00007D0022907D003299D
:1013200007D0042907D0002070470220704704200E
:10133000704700797047407970470000B42700007B
:1013400010B5FFF7C0FF04210348FFF72FFF024944
:101350000120487210BD00003C0000202DE9F0473C
:101360008CB0FFF711FB18B100200CB0BDE8F0877E
:10137000784C0020C4F81804BFF34F8F60680290C7
:10138000A5684FF00008284004EB800008E02168C1
:101390000298814201D86160E6E7284004EB8000B2
:1013A0000C3002A9FFF798FB0028F0D103AB02999B
:1013B00001EA050204EB8202491CD26843F82020AE
:1013C000401C02910228F2D3039800F00300022887
:1013D00002D001284ED0A5E003985022810D894605
:1013E000B2EB905F00D850210E4666F39F500390F9
:1013F0000831594800F01FFA070078D000F064FA6D
:101400004346082203A9384600F079FA029908F108
:10141000080A2940681A8000001D864223D94D4DD4
:101420000C3530B1C2B204EB8101301A90460C3158
:1014300004E02946F2B2002590462846C6B253463B
:10144000384600F05CFA0AEB08032DB13246294613
:101450004FEA070000F053FA029909F1030001EB8B
:10146000900002903AE004EB810153463246384640
:101470000C31EFE70398C0F38311062900D306214E
:1014800061F389100390C0F38310801C81003248FF
:1014900000F0D1F9070045D000F016FA43460822C3
:1014A00003A9384600F02BFA08F1080800260FE0DF
:1014B0000298434600EA0501401C04EB81010290BA
:1014C000042238460C3100F01AFA08F10408761CA0
:1014D0000398C0F38310B042EAD847B1D4F810544F
:1014E000D4F8180468B1384600F0F4F92CE019E09B
:1014F000687A012804D12A6828463946126890473C
:101500006D68002DF4D1384600F0E4F90020FFF7B3
:1015100048F9D4F8180408B9029860600020FFF771
:1015200042F911E0D4F8104404E0216820468968AB
:1015300088476468002CF8D108480221008801EB34
:10154000004007A100F06AF8FFF71EFA80F00100E2
:101550000BE700005C020020F4270000B800002028
:101560004261636B656E647320666C757368656455
:10157000000000002DE9F84F8146DFF89C80D01C68
:1015800015468A46800800226946D8F80860FFF7A9
:10159000A7F9B8B3009CA01C0090D8F80810304000
:1015A000091A8F003F1DBD4208EB800002D82A4671
:1015B000514608E03A4651460C30FEF7B3FE164855
:1015C000EA1B0AEB07010C30FEF7ACFE4FEA1947A5
:1015D000FFF7E4F947EA0042601C304008EB800066
:1015E000344008EB8401C260C8684FF6C07269F3EA
:1015F000C500904365F39F5020F00300801C20F04D
:101600000400C86098F8200402E000BFFFF7A6FEBF
:101610000028FBD1BDE8F88F5C02002000231A46A9
:1016200000F0C8BD2DE9F0470E4680461C469246A4
:1016300008293ED894F80C900020207319461046D3
:1016400000F0D0FC0025B54206D218F805201AA1FA
:101650002046FFF749FC03E019A12046FFF744FCB0
:101660006D1C082DEFD317A12046FFF73DFC002588
:10167000B54210D218F80570FEF750FE0068C05D44
:1016800010F03E0F01D03A4600E02E220EA1204677
:10169000FFF72AFC03E00DA12046FFF725FC6D1C97
:1016A000082DE5D301222146504600F07DFC84F848
:1016B0000C90BDE8F0870000202530327800000053
:1016C000202020007C000000256300002000000096
:1016D000104810B5FF218160002101604160C0F811
:1016E0001814C0F8141480F820140B4800F0F0F817
:1016F00000280DD109480A490A4B401AC1080020A8
:1017000003E000BF23F82000401C8842FAD30020E9
:1017100010BD00005C020020F4270000F427000048
:10172000B42700009C00002002480349401AC0086A
:1017300070470000F4270000B427000013B5684686
:10174000FFF7E2FA08B100201CBD0248009950F8EA
:1017500031001CBDB427000070B508480125D0F841
:10176000104480F8205405E06572216820464968DD
:1017700088476468002CF7D170BD00005C0200202F
:101780002DE9FF4781460C9D00200C462F7B2873D6
:10179000984616462946184600F024FC072E42D2E9
:1017A000DFE806F004090F161F2A360049462846CE
:1017B000FFF79AFB37E0494628462268FFF794FB7B
:1017C00031E0D4E9002349462846FFF78DFB2AE0A3
:1017D000A0680090D4E9002349462846FFF784FB1F
:1017E00021E0D4E90201CDE90001D4E90023494612
:1017F0002846FFF779FB16E004F1080007C88DE8DA
:101800000700D4E9002349462846FFF76DFB0AE0AC
:1018100004F108000FC88DE80F00D4E90023494601
:101820002846FFF761FB00222946404600F0BCFB3A
:101830002F73BDE8FF872DE9F041858A80462D1F73
:101840004819C01CB0FBF5F0C6B24046FFF796FA47
:10185000041E19D00020207101206071E58000274E
:101860002546761EC4F800800BE04046FFF786FA56
:1018700060B16179491C6171286005467F1CC0F820
:101880000080B742F1D32046BDE8F081204600F049
:1018900002F80020F8E72DE9F041457901466B1E7A
:1018A000002201E00968521C9A42FBD30F680146EE
:1018B000002605E038460C68FFF77FFA2146761CC3
:1018C000AE42F7D3BDE8F0810121001DFFF73ABA1F
:1018D000FFF788BA10B504460121001DFFF748FA4A
:1018E00010F0FF0F04D12046BDE81040FFF7D3BF32
:1018F00010BD38B501240094FFF7CAF938BD38B5DA
:1019000000240094FFF7C4F938BD01680A684968EB
:101910008068884201D9491C00E00021914201D130
:1019200001207047002070478068884201D9481C18
:101930007047002070472DE9F04104464FF0000841
:101940000E464046FEF72DFF2046FFF7DEFF07005C
:1019500009D0207C38B14FF004080020FEF723FFA7
:101960004046BDE8F0812068456841682046FFF7A1
:10197000DBFF2168486037B1206801682046FFF727
:10198000D3FF21680860E268012A14D0022A16D029
:10199000042A19D0082A1CD06068314605FB0200D1
:1019A000FEF7C0FC204600F0A8FB21688A6882424E
:1019B000D3D28860D1E7616830784855F2E7616832
:1019C000308821F81500EDE76168306841F825009E
:1019D000E8E7D6E90001626802EBC502C2E900014E
:1019E000E0E72DE9F04107464FF0000415000E46F0
:1019F000204611D0FEF7D5FE384600F07EFBA84207
:101A000005D32A463146384600F044FB00E0052461
:101A10000020FEF7C8FE2046BDE8F08110B5044660
:101A20000020FEF7BEFE204600F067FB04460020C3
:101A3000FEF7B9FE204610BD4058002800D0012016
:101A4000704708B5002242504058009008BDD0F8B9
:101A50000403084000D0012070474058002800D0FF
:101A60000120704708B5002242504058009008BD40
:101A70000121B1EB507F01D1012070470020704758
:101A800070B50D4600F0FAFA04000FD00020FEF702
:101A900088FE207920B10020FEF785FE112070BD60
:101AA0000120256020710020FEF77DFE002070BD22
:101AB00010B500F0E3FA002802D0002101600171A6
:101AC00010BD000001B569460548FFF734FF044822
:101AD000FFF71BFF002801D000F042F808BD00000E
:101AE0000C280000124A13780BB185207047516012
:101AF0000178C90704D00F490B6843F001030B605C
:101B00000D49D1F8003223F00103C1F800324078CA
:101B10000A49400181F8000401234FF0E0205903F5
:101B2000C0F88012C0F80011137000207047000048
:101B30001800002004D5004000D000400DE000E077
:101B4000064908B5002204480A600968009101218D
:101B5000C0F80413016008BD00D0004000D100406F
:101B600003490120C1F80803091D086070470000FF
:101B700000D000400149024800F0C6BB0C01002023
:101B8000002000402DE9F0410546007916460F4639
:101B900000EB40012D4A01EBC00102EB810494F8F7
:101BA0002A1011B10820BDE8F081294951F8201010
:101BB0002868FFF765FF08B11120F4E73946284689
:101BC000FEF706FE66603869206030004FF00106BF
:101BD0002FD03F7F4FF48E712868FFF732FF4FF40C
:101BE000A2712868FFF72DFF28681A49C0F804136E
:101BF00028684FEA4711000B40B2002806DA00F0CF
:101C00000F0000F1E02080F8141D03E000F1E02057
:101C100080F800142868000B40B200F01F0206FA9A
:101C200002F14009800000F1E020C0F88012C0F805
:101C3000001128680421C0F800150020A061E061AF
:101C400084F8290044F8140FA675ACE70C010020B5
:101C500018260000800002002DE9F04705460079B3
:101C60000B4600EB400101EBC000234901EB80046F
:101C7000284600F043F810B11120BDE8F0874FF07E
:101C80000008C4F82080A360626184F828804FF4C3
:101C90008E76474631462868FFF7D3FE28684FF016
:101CA0000109C0F808902146286800F0C9FA606868
:101CB00000BBD5F800A00EE094F8280008B10F276B
:101CC00016E031465046FFF7B7FE0028F4D0214613
:101CD000504600F0B5FA216A60698142F1D331467D
:101CE0002868FFF7A9FE0028F9D02868C0F80C90F2
:101CF000C4F814803846C0E70C010020007900EBDE
:101D0000400101EBC000044901EB8000406900285C
:101D100000D00120704700000C0100202DE9F047A1
:101D2000044600794FF0000900EB400101EBC000D0
:101D3000254901EB80072068C0F80095786880B1DC
:101D400020682249C0F8081320680121000B40B226
:101D500000F01F0291404009800000F1E020C0F82F
:101D600080112068D0F80C25D0F81485D0F80865CB
:101D7000D0F810554FF0FF31C0F81415C0F80C150D
:101D80002068C0F80815C0F81015501C02D0104685
:101D9000FFF7D4F9B8F1FF3F02D04046FFF7CEF984
:101DA000681C02D02846FFF7C9F9701C02D03046E3
:101DB000FFF7C4F92068FFF77BFE87F82A90C7F881
:101DC0000490BDE8F08700000C01002084020200AE
:101DD0000149024800F044BB3801002000200040C7
:101DE0002DE9F0410546164600790F46154A00EBED
:101DF000C00102EB810494F8201011B10820BDE865
:101E0000F081114951F820102868FFF739FE08B118
:101E10001120F4E739462846FEF71EFD6660386952
:101E200020601EB1397F2846FEF716FE286808217B
:101E3000C0F800150020A061E0610121606184F814
:101E40002010DCE7380100201C2600002DE9F047B7
:101E500004460E460079204900EBC00001EB8005E6
:101E600017463046FFF704FE30B1204600F036F842
:101E700020B11120BDE8F0871020FBE76F61AE6054
:101E80004FF49076002731462068FFF7EBFD4FF4C2
:101E9000AC7841462068FFF7E5FD2068AA686969CB
:101EA000C0F84425C0F848152068012181606868A1
:101EB00078B9B14649462068FFF7CFFD064641464E
:101EC0002068FFF7CAFD0643F4D000B10F270020B9
:101ED00068613846CEE700003801002000790549E6
:101EE00000EBC00001EB80004069002800D0012019
:101EF00070470000380100202DE9F04704460079C2
:101F0000274900EBC00001EB800720684FF0000973
:101F1000C0F80095786880B120682249C0F808139D
:101F200020680121000B40B200F01F0291404009DF
:101F3000800000F1E020C0F880112068D0F80C2566
:101F4000D0F81485D0F80865D0F810554FF0FF315F
:101F5000C0F80C15C0F814152068C0F80815C0F8B2
:101F60001015501C02D01046FFF7F1F8B8F1FF3FF2
:101F700002D04046FFF7EBF8681C02D02846FFF776
:101F8000E6F8701C02D03046FFF7E1F82068FFF752
:101F90008FFD87F82090C7F80490BDE8F087000017
:101FA000380100201003020010B50C46017A052903
:101FB00008D0407A38B1084808A102682046FEF7E8
:101FC00093FF00E01AB106A12046FEF78DFF2046E0
:101FD000BDE81040FEF795BF740000202573000097
:101FE0000D0A000038B5C3880D46044633B114A06D
:101FF000009015A216A12846FEF776FF217A052942
:102000001CD0607A48B1A088FFF782F9164951F8D0
:10201000202016A12846FEF767FFA0880021FFF7C1
:102020008DFB03461049207A143951F8202001B065
:102030002846BDE830400EA1FEF756BF38BD00006F
:102040001B5B306D000000001B5B313B33316D00CA
:1020500025734C6F67732064726F707065642028FD
:1020600025642925730D0A007400002025730000E3
:102070003C25733E2025733A200000000349884226
:1020800001D1034870470020704700000020004045
:10209000100000202DE9F0410446006817468846EC
:1020A00005684068854201D8461B02E0A068461BCF
:1020B000761CE2686068B74205FB02010CD87A43DF
:1020C0004046FEF72FF9A168E819884200D90020A0
:1020D00021680860BDE8F08102FB06F52A4640460B
:1020E000FEF720F9E268BE1B724308EB0500616849
:1020F000FEF718F920680660ECE701680A6849688D
:10210000914201D3881A70478068801A0844401CA5
:10211000704770B5054688690C4600284FF48471F5
:1021200028460AD0FFF78DFCD5F81805626AE168E9
:102130008854606A401C606270BDFFF782FCD5F86D
:10214000180570BD1FB501238DF80030CDE90121C0
:10215000D0E90012684690471FBD1FB501238DF8D6
:1021600000308DF808100192D0E9001268469047BF
:102170001FBD000070B50D4C0020D2B22070201D94
:102180000B4D0378EB5C1BB1001DFFF75FFE02E017
:102190000C30FFF761FD08B1FEF7F8FA607800280F
:1021A00002D021780029FAD070BD00002400002060
:1021B000040000202DE9F84F204D9246894606463E
:1021C0009846012269461846AF68FEF789FB58B366
:1021D000009800210446801C09E000BF00EA0703C4
:1021E0005AF8212005EB8303401C491CDA60414565
:1021F000F4D34FEA164AFEF7D1FB4AEA0041601CCD
:10220000384005EB80003C4005EB8402C160D0689B
:1022100066F3C50068F3891069F39F2020F003007E
:10222000401C20F00400D06095F8200402E000BFBC
:10223000FFF794F80028FBD1BDE8F88F5C0200207E
:1022400070B50C4605464FF48E71FFF7FAFB216A14
:10225000A068415C206A401C2062C5F81C1570BD56
:102260001FB500228DF80020029181680191426122
:10227000D0E90012684690471FBD00001FB50A460E
:1022800001788DF8001041680191017A8DF80810ED
:10229000C0680390044850F82210001F50F8222014
:1022A000684690471FBD00000C0000200149012036
:1022B000087070472400002010B588B00446202222
:1022C0000E496846FEF72EF806200090C01F0190C8
:1022D000029003904FF0EB7006900CB1084A00E0BA
:1022E000002269460748FEF7CBFD08B1FEF74EFA1B
:1022F0000448001F447008B010BD00003C260000D8
:10230000AD220000280000202DE9FF470C460546BD
:102310004FF40071FFF79BFB01274FF40178002673
:1023200018B34FF4927949462846FFF785FBE0B190
:1023300049462846FFF785FBC5F8088394F829002D
:1023400000B96F6002208DF80000D5F88004C5F850
:1023500080040390A0690290E0680190A661E661A4
:10236000D4E900126846904728E004212846FFF788
:102370006EFB18B34FF484712846FFF75DFBE8B19C
:1023800021462846FFF7C5FE616AA069884215D13B
:10239000E06938B1E268616AA0612069E66166625D
:1023A000E06008E094F8290000B96F60C5F8088380
:1023B000A661E268616A2046FFF7C4FE4FF48E789A
:1023C00041462846FFF738FB78B1206A61698842A8
:1023D00002D294F8280020B341462846FFF731FB8B
:1023E000616911B12046FFF73BFF4FF4A2784146E7
:1023F0002846FFF721FB002818D041462846FFF762
:1024000020FB94F8290000B12F60A06900280DD0AE
:10241000A661E268616A04B02046BDE8F047FFF7B4
:1024200091BE21462846FFF70BFFDEE7BDE8FF8798
:102430001FB50A4601788DF8001041680191017AB4
:102440008DF80810C0680390044850F82210001F4F
:1024500050F82220684690471FBD00000C00002065
:102460002DE9FF410C464FF4927705463946FFF7B8
:10247000F4FA0026C0B139462846FFF7F3FA0220E5
:102480008DF80000D5F88004C5F880040390D5F8D5
:102490003C058DF80800E0680190A661E661D4E98A
:1024A00000126846904723E04FF488773946284663
:1024B000FFF7D3FAE0B139462846FFF7D3FAD5F84B
:1024C0003C15A069884213D1E06960B1E268D5F893
:1024D000000220F02000C5F80002E069A061206938
:1024E000E661E06001E0A661E2682046FFF735FEA4
:1024F0004FF4A27739462846FFF7AFFA60B1394664
:102500002846FFF7AFFAA06930B1A661D5F83C15AF
:102510002046E268FFF721FE4FF4907739462846BF
:10252000FFF79BFA002813D039462846FFF79AFA9E
:10253000606900280CD0D5F84C058DF800608DF846
:102540000800A06801906661D4E9001268469047CF
:10255000BDE8FF812DE9F05F8346DDE90A4A99462F
:1025600090460D460846012703E000BFB0FBF8F097
:102570007F1C4045FAD2B94500D94F465FEACA7080
:1025800012D18CB15FEA8A7002D5B9F1000F01D087
:10259000202607E0302605E031465846641EFEF747
:1025A000E3F90CB1A742F7D35FF00106B9F1010FCF
:1025B00002D9A9F1010903E0B5FBF6F0404502D3C9
:1025C00006FB08F6F2E7DFF83C9000BFB5FBF6F03B
:1025D00000FB165519F800105846FEF7C5F9B6FB72
:1025E000F8F6002EF2D15FEACA7009D0002C07D0AD
:1025F000A74205D220215846641EFEF7B5F9F5E73B
:10260000BDE8F09F20260000000000000000000050
:102610000338FDD870470107751B0000D11D00006D
:102620003031323334353637383941424344454608
:10263000F9120000CD120000C5120000FFFFFFFFDD
:10264000FFFFFFFFFFFFFFFFFFFFFFFF0000000096
:10265000000000000000D6010701000000404040DB
:102660004040404040404141414141404040404065
:102670004040404040404040404040404005020211
:1026800002020202020202020202020202202020D0
:10269000202020202020200202020202020290902C
:1026A000909090901010101010101010101010102A
:1026B000101010101010101002020202020288887E
:1026C000888888880808080808080808080808088A
:1026D0000808080808080808020202024000000072
:1026E0005D2600007761726E696E670064656275D1
:1026F000670000001B5B313B33306D001B5B306DAE
:10270000000000001B5B313B33316D001B5B313B34
:1027100033326D001B5B313B33336D001B5B313B50
:1027200033346D001B5B313B33356D001B5B313B3C
:1027300033366D001B5B313B33376D00696E666F5E
:10274000000000006572726F72000000726E670018
:1027500071756575652E6D5F72616E645F706F6F08
:102760006C00000050525300524E470055415254E5
:1027700000000000554152544500000062616C6C3D
:102780006F632E6C6F675F6D656D706F6F6C0000AF
:10279000617070002428000000000020BC000000D0
:1027A000F0060000E0280000BC000020C425000066
:1027B000000700004C270000000000005027000028
:1027C00000000003642700000000000068270000EC
:1027D000000000006C2700000000000074270000CB
:1027E000000000007C27000000000003902700008C
:1027F000000003035000002048000020500000208B
:102800009C010020B40000201800000000010020FE
:10281000BC0000204000000001000000000000009B
:10282000A0000020000000000000000000000000E8
:102830000000000000000000000000000000000098
:102840000000000000000000000000000000000088
:1028500000200040000000000020004000000000B8
:102860003026000000000000000000000000000012
:102870000000000000000000000000000000000058
:10288000000000000000000044270000E4260000D3
:102890003C270000EC260000FC260000F426000087
:1028A000042700000C270000142700001C2700004C
:1028B000242700002C270000342700000090D003BC
:1028C0000000000000000000000000000000000008
:1028D00000000000000000000000000000000000F8
:0400000500000201F4
:00000001FF
